:100000000C9429050C9470050C9470050C944A26E8
:100010000C9470050C9470050C9470050C9470058C
:100020000C9470050C9470050C9473230C94492463
:100030000C94CC130C9470050C9470050C94700502
:100040000C9470050C9470050C9470050C9470055C
:100050000C9470050C944F230C9470050C9470054F
:100060000C9470050C9470050C9470050C9470053C
:100070000C9470050C9470050C9470050C9470052C
:100080000C9470050C9470050C9470050C9470051C
:100090000C9470050C9470050C9470050C9470050C
:1000A0000C9470050C9470050C9470050501098082
:1000B000A101850319012AB700150126B700950192
:1000C00075108100C0050C0901A101850419012AE0
:1000D000A002150126A002950175108100C00660DE
:1000E000FF0961A1010962150026FF00952075082E
:1000F00081020963150026FF00952075089102C052
:1001000005010906A101050719E029E715002501E8
:10011000950875018102950175088101050719008F
:1001200029FF150026FF00950675088100050819AE
:10013000012905950575019102950175039101C08D
:1001400000AF09025B00030100A0FA0904000001EE
:10015000030101000921110100012240000705816E
:100160000308000A0904010002030000000921112C
:100170000100012222000705820320000107050378
:1001800003200001090402000103000000092111FD
:100190000100012232000705840320000A12010039
:1001A0000200000008C58E58010100010200011084
:1001B000034C006F007400750073003500380000B8
:1001C000001C034C006F00720064004F0066005377
:1001D00000610072006300610073006D00000004A4
:1001E00003090407087F0807003E5B4F5B3E003EA3
:1001F0006B4F6B3E001C3E7C3E1C00183C7E3C1846
:10020000001C577D571C001C5E7F5E1C0000183CC4
:10021000180000FFE7C3E7FF00001824180000FFE4
:10022000E7DBE7FF0030483A060E00262979292649
:1002300000407F05050700407F05253F005A3CE749
:100240003C5A007F3E1C1C0800081C1C3E7F00140A
:10025000227F2214005F5F005F5F0006097F017F3D
:1002600000006689956A0060606060600094A2FF8B
:10027000A2940008047E04080010207E20100008CC
:10028000082A1C0800081C2A0808001E101010105C
:10029000000C1E0C1E0C0030383E383000060E3E9E
:1002A0000E060000000000000000005F00000000DB
:1002B0000700070000147F147F1400242A7F2A12ED
:1002C00000231308646200364956205000000807D6
:1002D000030000001C224100000041221C00002AF3
:1002E0001C7F1C2A0008083E0808000080703000AF
:1002F00000080808080800000060600000201008DE
:100300000402003E5149453E0000427F4000007219
:1003100049494946002141494D33001814127F10C4
:10032000002745454539003C4A49493100412111E2
:10033000090700364949493600464949291E000047
:1003400000140000000040340000000008142241A6
:10035000001414141414000041221408000201595E
:100360000906003E415D594E007C1211127C007F4F
:1003700049494936003E41414122007F4141413EC9
:10038000007F49494941007F09090901003E414177
:100390005173007F0808087F0000417F4100002062
:1003A00040413F01007F08142241007F404040400F
:1003B000007F021C027F007F0408107F003E414145
:1003C000413E007F09090906003E4151215E007F40
:1003D000091929460026494949320003017F0103D2
:1003E000003F4040403F001F2040201F003F40385A
:1003F000403F0063140814630003047804030061A1
:1004000059494D4300007F4141410002040810203A
:1004100000004141417F00040201020400404040CD
:100420004040000003070800002054547840007F3B
:100430002844443800384444442800384444287F41
:100440000038545454180000087E09020018A4A46F
:100450009C78007F080404780000447D4000002060
:1004600040403D00007F102844000000417F4000D4
:10047000007C04780478007C080404780038444444
:10048000443800FC182424180018242418FC007C8C
:10049000080404080048545454240004043F44242D
:1004A000003C4040207C001C2040201C003C403090
:1004B000403C004428102844004C9090907C00441C
:1004C00064544C44000008364100000000770000EE
:1004D000000041360800000201020402003C26230D
:1004E000263C00000000000000404040F0F8F8FF0B
:1004F00038FFF8F83FF8F8FF38FFF8F8F0404040D0
:1005000000000000000080C0C0C0800000C0C080AB
:1005100000000080C0C000C0C0000080C0C000005B
:10052000000000C0C0C0C0C000C0C000000000008B
:1005300000000000000000000000000000000000BB
:1005400000000000000000000000000000000000AB
:10055000000000000000000000000000000000009B
:100560000000C0F0F8FC3E1E06010000007F414183
:10057000417F007F4141417F000080C0E07E5B4FB2
:100580005BFEC00000C000DCD7DEDEDED7DC00C0D2
:10059000000000000000000000000000000000005B
:1005A000000000000000000000494949FFFFFFFF74
:1005B000E0DFBFBF00BFBFDFE0FFFFFFFF494949EA
:1005C00000000000001F3F6060E0BF1F007F7F074A
:1005D0001E381E077F7F007F7F0E1F3B716000006B
:1005E0000000007F7F0C0C0C007E7E007F7E0303EA
:1005F000007F7E03037E7E03037F7E000F3E703C00
:10060000063C703E0F00327B49493F7E007F7E03EF
:1006100003001E3F69696F26000000000000000013
:100620000000030F1F3F3C7870600000007F4141D5
:10063000417F007F4141417F00307B7F7830202027
:1006400030787F3B0003000F7F0F0F0F7F0F0003F9
:10065000000000000000000000000000000000009A
:10066000000000000000000000010101070F0F7FE3
:100670000F7F0F0F7E0F0F7F0F7F0F0F07010101FD
:100680000000000000000000000001010000000068
:10069000000000000000000000000000000000005A
:1006A000000000000000000000000000000000004A
:1006B000000000000000000000000000000000003A
:1006C000000000000000000000000000000000002A
:1006D000000000000000000000000000000000001A
:1006E000000000000000000000000000000000000A
:1006F00000000000000000000000000000000000FA
:1007000000000000000000000000000000000000E9
:1007100000000000000000000000000000000000D9
:1007200000000035001E001F0020002100220029CB
:100730000014001A000800150017002B0004001612
:1007400000070009000A00E1001D001B0006001957
:10075000000500E300E200E00002512800A8003597
:1007600000270026002500240023002A0013001281
:10077000000C0018001C00340033000F000E000DA8
:10078000000B00E50038003700360010001100E7CC
:1007900000E600E40003512C00000035001E001F9D
:1007A00000200021002200290014001A0009001373
:1007B000000A002B0004001500160017000700E1D6
:1007C000001D001B00060019000500E300E200E028
:1007D0000001002800A8003500270026002500247D
:1007E0000023002A0033001C0018000F000D003405
:1007F0000012000C00080011000B00E50038003763
:1008000000360010000E00E700E600E40001002CB6
:1008100000000001003A003B003C003D003E003576
:10082000001E001F0020002100220001001E021FE8
:100830000220022102220201002E002D002E022F92
:10084000023002010001000100010001000100442A
:100850000043004200410040003F004500270026C1
:10086000002500240023003102270226022502244D
:10087000022302010031003302330030002F000157
:100880000001000100010001000100010001000160
:100890000001000100010001004900460065000060
:1008A0000000000100E200E000E10000003900016A
:1008B000007A007B007C007D000000010001000147
:1008C0000001000100010001000100010001000120
:1008D0000001002A0001000100520001004B002A23
:1008E000004C004F00510050004E0001000000017C
:1008F00000000001000000010001000100010001F2
:1009000000010000DA0281FFD9F1DB20A4A62EAF9E
:1009100000A0C000A1C800AED580A81FD300408DA4
:100920001420004350534C4B000A0A00556E646576
:1009300066004C6F776572005261697365004261B1
:1009400073650A004C41594552000A0A004D6F6414
:100950000A00436C6D6B0051777274000A0A0080C4
:100960008182838485868788898A8B8C8D8E8F90FF
:1009700091929394A0A1A2A3A4A5A6A7A8A9AAAB6B
:10098000ACADAEAFB0B1B2B3B4C0C1C2C3C4C5C6E2
:10099000C7C8C9CACBCCCDCECFD0D1D2D3D400001A
:1009A000AE00000000000000000000000000000099
:1009B0000000000000000000000000000000000037
:1009C00000000000007E0F00D4FFFFFFC700000002
:1009D0007800000000000000002A2B280000000022
:1009E00000000000000000000000000029000000DE
:1009F000002C1E3420212224342627252E362D3784
:100A000038271E1F202122232425263333362E3754
:100A1000381F0405060708090A0B0C0D0E0F1011EC
:100A200012131415161718191A1B1C1D2F313023F9
:100A30002D350405060708090A0B0C0D0E0F1011C1
:100A400012131415161718191A1B1C1D2F313035C7
:100A50004C0011241FBECFEFDAE0DEBFCDBF04B6DD
:100A600003FE27C08091E8049091E904A091EA0474
:100A7000B091EB048730904BA740B04BD1F410926B
:100A8000E8041092E9041092EA041092EB0414BEF8
:100A900084B7877F84BF0FB6F894A89580916000D3
:100AA000886180936000109260000FBEE0E0F8E380
:100AB000099511E0A0E0B1E0E2E4F1E502C00590A3
:100AC0000D92A23DB107D9F724E0A2EDB1E001C03B
:100AD0001D92A83EB207E1F70E94A11D0C94672861
:100AE0000C940000982F82958F7011F0982F84E05D
:100AF000292F2695269511F08E5F922F969509F055
:100B00008F5F0895E92FEE0FE90FEE0FE80F8E2F9C
:100B1000877041E001C0440F8A95EAF7E695E695B3
:100B2000E69583E0E89FF0011124E357FB4F30E0A6
:100B300020E070E05191DF011197CB01022E02C03D
:100B4000969587950A94E2F781708195852784238D
:100B500085278C932F5F3F4F2330310559F7089538
:100B6000E92FEE0FE90FEE0FE80F9E2F9770E69535
:100B7000E695E69583E0E89FF0011124E357FB4FEB
:100B800050E040E080E0219130E0092E02C036952F
:100B900027950A94E2F721703327042E01C0220F13
:100BA0000A94EAF7822B4F5F5F4F4330510559F7A4
:100BB00008958091B1049091B004981301C00895F4
:100BC0008F5F8770FACFE7EDF1E09191891303C051
:100BD000DF0111971C9291E0ED3DF907B1F70895FF
:100BE0008091A90481111092A90408958091A8040C
:100BF0009091AF04892B9091A504892B8093D50106
:100C00009091A904992391F0892B8093D50120E03C
:100C100087ED91E0FC013081019631112F5F31E0C9
:100C20008D3D9307B9F721110E94F005E0918B04E7
:100C3000F0918C04309731F00280F381E02D85ED46
:100C400091E009940895882339F09091A804892BA4
:100C50008093A8040C94F6050895882341F08095AC
:100C60009091A80489238093A8040C94F605089514
:100C70009091AC0492FF06C0282F28712830F9F417
:100C8000877F846093FF06C0282F28712831F1F4F4
:100C9000877E84612091AD0420FF06C0382F387113
:100CA0003830D9F4877F816021FF06C0282F287152
:100CB0002831D1F4877E816194FD877E0895282FA5
:100CC00024712430F9F68B7F8860DCCF282F2471C3
:100CD000243101F78B7E8861DDCF382F31713130BF
:100CE00019F78E7F8860E0CF282F2171213121F7FD
:100CF0008E7E8861E1CFCF93DF93EC01803E91053A
:100D000009F45EC048F58133910509F4A1C088F467
:100D10008932910509F495C08A9709F4A0C0C130C1
:100D2000D10529F1CE010497813A910508F054C00C
:100D30001EC089339105E9F182389105D1F1C5973B
:100D400009F478C0C83AD10508F090C0C53AD10579
:100D500030F3A497D0640BC0843E910509F44FC0D2
:100D600050F4823E9105D9F1833E9105E9F1CE011F
:100D7000DF91CF910895863E910509F44BC0873EDF
:100D8000910509F44CC0811523E5920708F08BC04A
:100D9000811532E5930708F0FDC0C11580E5D8073D
:100DA00008F077C0C11520E4D20760F2DF70D06A86
:100DB000DECF8091AC048370D1F2C0EED0E0D7CF0B
:100DC0008091AC0480FD11C19091AD0490FFCFCF14
:100DD000C3EED0E084FFCBCFD0E0C0E0C8CF80919D
:100DE000AC0482FDF5CFC3CF8091AC0482FD00C17D
:100DF0009091AD0490FDE1CF84FFB9CFEDCF80910C
:100E0000AD0481FFB4CF8091AC04C7EED0E084FD87
:100E1000E3CFADCF8091AC0483FDF7CFA8CF809115
:100E2000AC0483FDE8C09091AD0491FFE5CFC4EE22
:100E3000D0E09DCF8091AC0485FF99CFC9E2D0E08E
:100E400096CF8091AC0485FF92CFC5E3D0E08FCFE1
:100E50008091AC0486FF8BCFCAE2D0E088CF80912E
:100E6000AC0486FF84CFC1E3D0E081CFCF3BD10576
:100E700008F468C0C83ED10528F4C03ED10508F486
:100E8000ABCF75CFCE019A9581159F4108F0A4CFC5
:100E90006ECFC11581E5D80708F45FC0DC2FCC27E1
:100EA000C16FD06A64CF811529E59207A0F581153D
:100EB00038E5930708F086C0C11585E5D807C8F462
:100EC000C11524E5D20708F078C09E0123703327AE
:100ED00081E090E002C0880F991F2A95E2F7C6953D
:100EE000C69530E2C39FE0011124C82BD92BDA68E4
:100EF0003ECFCE0195558F3F910511F008F06CCF94
:100F00008C2F0E943806C82FD0E0DC2FCC27CC27AE
:100F1000DF71D0622CCFC1158AE5D80708F457C01D
:100F2000CE0190568115904208F056CF8D2F8F71CB
:100F30000E94380690E0982F882788279F718C2B75
:100F4000EC01E7CFC85AD0E0CC0FDD1FCC55DE4F07
:100F50000990D881C02DD4640ACF9E0174E03695E3
:100F600027957A95E1F723708C2F86958695837067
:100F700030E2839FC0011124922BC37021E030E046
:100F800002C0220F331FCA95E2F7822B932BEC018C
:100F9000DC68EDCE9C012370332781E090E002C035
:100FA000880F991F2A95E2F7C695C69520E2C29F41
:100FB000E0011124C82BD92BEBCFDC2FCC27C46F39
:100FC000D06AD5CED82FCC27C06FD06AD0CE8C2F88
:100FD0008F700E94380634E0D695C7953A95E1F7B0
:100FE000CF709C2FEC01D069C2CEC9E3D0E0BFCE58
:100FF000C2EED0E0BCCEC6EED0E0B9CE80E008951F
:10100000F894E82FE295EF70F0E041A18F7021E0B5
:1010100030E0B90102C0660F771F8A95E2F7CB0175
:10102000962F9095942391A392A1892B82A37894D3
:101030000895FC01680F791F8FEF91E321918227BA
:1010400028E030E087FF09C0880F89272150310947
:10105000C9F7E617F70791F70895880FF7CF2091A2
:10106000F9013091FA012817390771F09093FA01CC
:101070008093F901E0918B04F0918C04309721F07A
:101080000680F781E02D099408952091F7013091B1
:10109000F8012817390771F09093F8018093F70150
:1010A000E0918B04F0918C04309721F00084F1855D
:1010B000E02D09940895882361F19CEF980F913AEF
:1010C00020F40E94E3050C94F60590E2980F983006
:1010D00088F4877021E030E0A90102C0440F551F59
:1010E0008A95E2F7CA0180959091A804892380939C
:1010F000A804E9CF9BE5980F933020F490E080E0BE
:101100000C942F08885A873120F490E080E00C94EA
:101110004508089590E080E00E942F0890E080E06C
:101120000E9445081092AF041092A5040C94F60595
:101130008093AA040C948A088093AB040C948A08C8
:1011400021E030E001C0220F8A95EAF78091AB04DC
:10115000822B0C949C0821E030E001C0220F8A957C
:10116000EAF720958091AB0482230C949C0890911F
:10117000AE04809589238093AE04282F277039F41C
:10118000282F082E000C330B9217130621F4909190
:10119000AD0492FF07C08595859585950E94AB08A3
:1011A0001092AE0408959C01FC0132968FEF90E0FE
:1011B0004191461751F08F3F19F4411101C0892F19
:1011C0009F5F9630A9F78F3F09F40895280F311DCE
:1011D00087FD3A95F90162830895CF93C82F88233C
:1011E00009F445C08CEF8C0F813A88F4E7EDF1E00B
:1011F0008191C817B1F121E0ED3DF207C9F76C2FDD
:1012000085ED91E00E94D308CF910C94F60580E221
:101210008C0F883068F4C77021E030E001C0220FE5
:10122000CA95EAF78091A804822B8093A804ECCF9A
:101230008BE58C0F833038F42C2F2452330BC901EB
:10124000CF910C942F08C85AC73188F4EC2FF0E0E6
:10125000EE0FFF1FEC55FE4F80819181CF910C94D2
:1012600045088C2F0E94E3050E94F605C8CFCF9158
:101270000895CF93DF9300D000D0CDB7DEB78FB7FE
:10128000F8942091520430915304409154045091A9
:10129000550429833A834B835C838FBF69817A81AC
:1012A0008B819C810F900F900F900F90DF91CF91C9
:1012B00008950C94390987E797E790930108809384
:1012C000000888E19AE00FB6F894A8958093600032
:1012D0000FBE90936000FFCF8091F60108950895AE
:1012E000FC01CB012091E9013091EA012617370773
:1012F00090F0009729F42091E8002E772093E800E1
:1013000040E0009751F4411108C08091E80082FF4D
:1013100031C080E00895C901F3CF209162042223F7
:10132000A9F12530A9F12091E80023FD2DC02091DD
:10133000E80022FDEACF2091E80020FFE2CF3091C3
:10134000F3002091F200009719F02830310558F091
:1013500041E02830310509F040E02091E8002E7787
:101360002093E800CECF41914093F10001972F5F89
:101370003F4FE9CF80916204882341F0853041F0EE
:101380008091E80083FFC1CF81E0089582E0089555
:1013900083E008958091E30187FF13C08091E80006
:1013A00082FF06C08091E8008B778093E80004C03C
:1013B000809162048111F2CF0895809162048823A4
:1013C000D9F38091E80080FFF8CF8091E8008E7714
:1013D000ECCF2091E4003091E50095E6A901209141
:1013E000EC00822F817020FF06C08091E80080FF12
:1013F00006C080E008952091E80022FD1AC0809187
:101400006204882389F0853089F08091EB0085FDA6
:101410000FC02091E4003091E50042175307F9F224
:101420009150E1F684E0089582E0089583E0089504
:1014300081E00895E8EDF0E080818E7F8083109256
:10144000E2001092DA001092E100A0EEB0E08C9180
:1014500081608C9380818F77808319BCA7EDB0E089
:101460008C918E7F8C9380818F7E80831092E2019D
:101470000895EF92FF920F931F93CF937C018B01FE
:101480000E94E909C82F811117C08091E80085FDED
:101490000BC08091E8008E778093E8000E94E909F4
:1014A000882399F3C82F08C0F70181917F018093A9
:1014B000F1000150110949F78C2FCF911F910F9125
:1014C000FF90EF9008958091AB04982F967096301E
:1014D00019F488600C949C08877FFCCF982F909318
:1014E000E900242F762F50E0891731F07091EC003D
:1014F0002091ED005091F00021FD06C09F5F9730D4
:1015000071F78093E90008953091EB003E7F3093AE
:10151000EB003091ED003D7F3093ED003091EB001A
:1015200031603093EB007093EC002093ED0050930A
:10153000F0002091EE0027FDE1CF0895CF92DF92D9
:10154000EF92FF920F931F93CF93DF93C8EDD0E0FC
:1015500088818F7E8883E7EDF0E0808181608083E1
:1015600084E082BF81E08093E20188818E7F88835E
:1015700002EE10E0F80110821092DA0081EEC82E1F
:10158000D12CF601108288818F77888388818068CA
:10159000888388818F7D888319BC109262041092A1
:1015A000E10110923F041092E00190EEE92EF12C3F
:1015B000F70180818B7F808388818160888342E00E
:1015C00060E080E00E946E0AF60180818E7F808359
:1015D000F801808181608083808188608083F70149
:1015E00080818E7F8083888180618883DF91CF9125
:1015F0001F910F91FF90EF90DF90CF9008950F9380
:101600001F93CF93C82F0AE010E0893311F400E54F
:1016100010E08C2F0E94ED088FE99FE00197F1F711
:1016200000C0000001501109B9F78C2FCF911F9114
:101630000F910C945B08811106C089EA611101C009
:101640008AEA0C94FF0A813029F48EE46111F9CF03
:101650008BE4F7CF089580916304811110C08091CD
:10166000D80080618093D8008AE18A95F1F700C0A4
:101670008091D90080FF0AC081E08093630481E0FB
:1016800090916304913009F080E0089582E08093A6
:1016900063040E941A0A10926204F1CF0E942B0B7D
:1016A000882351F0E0918B04F0918C04309721F065
:1016B0000190F081E02D099480E00895AF92BF92EF
:1016C000CF92DF92EF92FF920F931F93CF93DF930E
:1016D000F82EE92ED62EC72E890180916704AA2400
:1016E000A394B12C8A3018F48AE0A82EB12CC1E062
:1016F000D0E0F8946D2D7C2D8F2D9E2DF80109954D
:101700007894811104C02196AC16BD065CF4DF917B
:10171000CF911F910F91FF90EF90DF90CF90BF90EE
:10172000AF900895CC9F9001CD9F300D300D1124C6
:1017300090E080E045E34A95F1F700000196281714
:101740003907C1F7D6CFCF93DF93D82FC92F81E0C8
:101750008093E9008FEF9091E800815095FD06C0DD
:1017600095ED9A95F1F700008111F5CF8091E80091
:1017700085FF16C050E040E068E070E08D2F9C2FA0
:101780000E94390A8091E8008E778093E80088E013
:10179000ED2FFC2FAEEEB1E001900D928A95E1F7AE
:1017A000DF91CF91089590916204943029F5809350
:1017B000EB016093EC017093ED019093E9008FEFE2
:1017C0009091E800815095FD06C095ED9A95F1F74E
:1017D00000008111F5CF8091E80085FF0DC050E039
:1017E00040E063E070E08BEE91E00E94390A809166
:1017F000E8008E778093E8000895BC0183E00C94A4
:10180000D30BBC0184E00C94D30BCF93C091AD04F7
:10181000C2FB992790F9981781F080FBC2F9C09319
:10182000AD046091AC0484E090E00E9433286C2FFA
:1018300082E290E0CF910C943328CF9108954F929B
:101840005F926F927F928F929F92AF92BF92CF9250
:10185000DF92EF92FF920F931F93CF93DF9310E0ED
:1018600000E038E7632E712CE801CC0FDD1F580132
:101870001CC0F60185909490692DC7010E94332801
:10188000682DC70101960E94332822E0C20ED11CA8
:1018900032E0E30EF11C4E145F0459F72C9686E0FB
:1018A000A80EB11CC615D70581F0C501880F991F78
:1018B0009C012D5D384F69017E0137E2E30EF11C7A
:1018C0002E0183E3480E511CD4CF3E0128E7620E5F
:1018D000711C045C1F4F003F110531F6DF91CF9161
:1018E0001F910F91FF90EF90DF90CF90BF90AF903E
:1018F0009F908F907F906F905F904F900895CF93BF
:10190000C82F6FEF811161E283E290E00E943328DB
:101910006FEFC11160E184E290E00E9433286FEF25
:10192000C11166E185E290E0CF910C943328CF930A
:10193000DF93C7E0D2E060E0CE010E943328219619
:10194000C11584E0D807B9F7DF91CF91089580E001
:101950000E947F0C60E086E290E00E9433280E94A3
:101960001F0C0E94970C81E00C947F0CCF9384E0B5
:1019700090E00E942528C82F82E290E00E9425284E
:10198000982F8C2FCF91089583E290E00E94252814
:10199000813289F484E290E00E942528803159F454
:1019A00085E290E00E94252891E0863109F090E0E0
:1019B000892F8170089580E0FCCF0F931F93CF9300
:1019C000DF93C42FD0E0CC0FDD1F2CE0629FC00D51
:1019D000D11D112438E7839FC00DD11D1124CE01E4
:1019E00087960E942528082F10E0102F0027CE018F
:1019F00088960E9425289801282BC901DF91CF9154
:101A00001F910F910895462F672F843030F47A305C
:101A100020F4463010F40C94DD0C90E080E0089542
:101A2000DF92EF92FF920F931F93CF93DF937C018E
:101A30000091AB048091AA04082BC7E0D0E010E02D
:101A4000DC2EC8010C2E02C0959587950A94E2F70A
:101A500080FD0CC02197A0F7D12C8D2DDF91CF9167
:101A60001F910F91FF90EF90DF900895B7018C2F99
:101A70000E94030D0E947B06019761F3EECF0F9346
:101A80001F93CF93FC01828100811181882389F00B
:101A9000662379F0C8010E94100DC82F682FC80175
:101AA0000E948205B8018C2FCF911F910F910C9449
:101AB000030DC8010E94B005C82FF4CFCF93DF9368
:101AC000D82FC92F0E94100D6D2F7C2F0E94030D5F
:101AD000DF91CF910C947B060E945E0D282F892FF9
:101AE0008F70392F32953F70903C80F43A30B0F4CB
:101AF000343020F4323090F480E008953630E1F74D
:101B000081E0283E88F0213FB9F70EC03C3011F04B
:101B10003F3091F7869586958695089581E0203F20
:101B200039F018F4283E40F70895243F29F7FCCFF8
:101B300008951092A804E7EDF1E086E0DF011D9220
:101B40008A95E9F70C948A081F93CF93DF93CDB75A
:101B5000DEB7AA970FB6F894DEBF0FBECDBF83EEF7
:101B600091E0FC0101962091F100208321E08B3E61
:101B70009207B9F78091E401893009F456C0C8F49E
:101B8000823009F4B2C0833009F481C0813071F130
:101B90008091E80083FF81C28091E3019091E4018C
:101BA0009A3008F07AC2E92FF0E0E759F74D0C942B
:101BB000F9278A3009F488C08B3051F78091E3010E
:101BC000813231F78091E7019091E801892B01F78B
:101BD0008091E800877F8093E8000E94CA09809185
:101BE000E501809300010E94990DD2CF8091E3011D
:101BF000813A71F68091E800877F8093E8008091B8
:101C0000E7019091E801892B61F468E08EEE91E0A4
:101C100070E00E9470098091E8008B778093E80063
:101C2000B7CF60E090E080E0F3CF8091E3018132B4
:101C300009F0AECF8091E7019091E8018D7F892B6B
:101C400009F0A6CF8091E800877F8093E80080911B
:101C5000E80082FF17C09091F3008091F200029794
:101C600029F48091F1008B7F813021F48091F10083
:101C70008093F6018091E8008B778093E8000E94C2
:101C8000CA0986CF809162048111E1CF81CF809112
:101C9000E301813A09F07CCF8091E7019091E8015E
:101CA000892B09F075CF8091E800877F8093E80049
:101CB0008091E80080FFFCCF809100018093F100CB
:101CC0008091E8008E77D9CF8091E301813209F0CD
:101CD0005FCF8091E800877F8093E8000E94CA0967
:101CE0008091E6018093DF0153CF8091E301813A37
:101CF00009F04ECF8091E800877F8093E8008091C3
:101D0000E80080FFFCCF8091DF01D8CF803899F0C8
:101D1000823809F0C2C18091E7018F70873008F0E6
:101D2000BCC18093E9008091EB0085FB882780F996
:101D30001092E90006C08091E00190913F0491115A
:101D400082609091E800977F9093E8008093F10083
:101D50001092F1008091E8008E779BC1882309F4EE
:101D600089C1823009F099C18091E50181118CC14E
:101D70008091E7018F702FEF280F263008F08DC17A
:101D80008093E9002091EB0020FF7EC1933031F475
:101D90008091EB0080628093EB0076C19091EB0024
:101DA00090619093EB0021E030E001C0220F8A9512
:101DB000EAF72093EA001092EA008091EB00886035
:101DC000EACF81116AC11091E5011F778091E3008C
:101DD0008078812B8093E3008091E800877F809357
:101DE000E8000E94CA098091E80080FFFCCF809142
:101DF000E30080688093E30082E0111183E0809328
:101E000062044BC18058823008F047C14091E5011F
:101E10005091E6014C3D83E0580799F583E08A83B1
:101E20008AE289834FB7F894DE01139620E03EE002
:101E300051E2E32FF0E050935700849120FF03C05C
:101E400082958F703F5F8F708A30C8F0895C90E018
:101E50008D939D932F5F243161F74FBF8091E800F0
:101E6000877F8093E8006AE270E0CE0101960E94CD
:101E700070098091E8008B778093E8000EC1805D47
:101E8000E6CF8091E7019091E801252F3327233099
:101E9000310509F44AC078F52130310509F479C0DB
:101EA0008BE590E0E2E4F1E02230310509F0F5C085
:101EB0002091E800277F2093E8002091E9013091EC
:101EC000EA018217930708F49C0140E021153105CF
:101ED00009F064C0411162C08091E80082FDC9CF61
:101EE00080916204882329F2853019F28091E800FC
:101EF00083FFF2CFBECF2132310509F43BC022323D
:101F0000310509F0CAC08330910508F0C6C0FC0154
:101F1000EE0FFF1FE259FE4F0190F081E02D855931
:101F20009E4FDC018C9190E011C0CA01992741308D
:101F300089F082309105B1F0892B09F0AEC0EFED48
:101F4000F1E0E4918E2F90E0EFEDF1E0009709F4DD
:101F5000A4C0AECFE1ECF1E0E4918E2F90E0E1EC93
:101F6000F1E0F4CFEFEAF1E0E4918E2F90E0EFEAB8
:101F7000F1E0ECCF8330910508F08FC0880F991FF6
:101F8000FC01EC58FE4F0190F081E02D89E090E0DB
:101F90008FCF82E190E0EDE9F1E08ACF8091620499
:101FA000882309F466CF853009F463CF8091E80077
:101FB00083FD5FCF8091E80082FD8ECF8091E800A5
:101FC00080FF84CF9091F3008091F20021153105BC
:101FD00019F08830910550F041E0089709F040E091
:101FE0008091E8008E778093E80070CF4491409311
:101FF000F1003196215031090196E8CF803809F07F
:102000004CC08091E800877F8093E8008091E101D7
:102010008093F1009FCE811140C01091E5011230F4
:10202000E0F58091E800877F8093E8001093E1015C
:102030000E94CA09112311F084E005C08091E300D9
:1020400087FDFACF81E08093620442E061EC81E099
:102050000E946E0A42E261EC84E00E946E0A42E253
:1020600061EC82E00E946E0A42E260EC83E00E9432
:102070006E0A13C08091E501813079F481E09330DC
:1020800009F080E080933F041092E9008091E8001D
:10209000877F8093E8000E94CA098091E80083FF4F
:1020A0000AC08091E800877F8093E8008091EB0070
:1020B00080628093EB00AA960FB6F894DEBF0FBE45
:1020C000CDBFDF91CF911F91089569EE7EEF90E033
:1020D00080E00E94512860E082E090E00E94332876
:1020E00060E083E090E00E9433281092AA0460E050
:1020F00084E090E00E94332860E082E290E00E9459
:10210000332860E085E090E00E94332860E086E0BC
:1021100090E00E9433286FEF87E090E00E94332820
:1021200040E050E0BA0188E090E00E94452860E07D
:102130008DE090E00E94332840E050E0BA0188E151
:1021400090E00E94452860E087E190E00E943328FB
:1021500040E050E0BA018CE190E00E94452870E038
:1021600060E080E290E00E94512840E050E0BA0137
:1021700088E190E00E94452880E00E947F0C0E9448
:10218000A70C40E050E0BA018FE090E00E944528A3
:1021900040E050E0BA0183E190E00C9445285F9262
:1021A0006F927F928F929F92AF92BF92CF92DF9267
:1021B000EF92FF920F931F93CF93DF930F92CDB7C0
:1021C000DEB7562E5A0149016701682E880F77083D
:1021D000C3010E941127892B09F089C08AE0869DDE
:1021E000F001879DF00D1124EB5EFE4F8581482F95
:1021F00050E0882311F041E050E08AE0869DF00134
:10220000879DF00D1124EB5EFE4F668177816A5A3F
:102210007B4FCE0101960E941C28D5014D915D9106
:102220006D917C912FB7F894809152049091530452
:10223000A0915404B09155042FBF841B950BA60B9D
:10224000B70B84369105A105B10540F4B601C8016C
:102250000E9419089981891709F450C0E52C550C82
:10226000FF08C7010E941127892B99F0F12C8F2DAF
:102270000F90DF91CF911F910F91FF90EF90DF9022
:10228000CF90BF90AF909F908F907F906F905F9016
:1022900008958AE08E9DF0018F9DF00D1124EB5E74
:1022A000FE4F458150E0C416D50608F4A6018AE029
:1022B0008E9DF0018F9DF00D1124EB5EFE4F668127
:1022C00077816A5A7B4FC4010E941C28B601C8015D
:1022D0000E94190899818913C9CF0E943909F50113
:1022E0006083718382839383FF24F394C0CFF12CA6
:1022F000A601B801C4010E941C28B9CFFF24F394A1
:10230000F7CFCF92DF92EF92FF920F931F93CF936D
:10231000DF9300D000D00F92CDB7DEB76B0185E020
:10232000E82EF12C07E514E09E012F5F3F4F4EE4AD
:1023300054E061E080E00E94CF10882349F095E0EE
:10234000FE013196A9E4B4E001900D929A95E1F76F
:1023500095E0E9E4F4E0D60101900D929A95E1F759
:102360000F900F900F900F900F90DF91CF911F91D2
:102370000F91FF90EF90DF90CF900895CF92DF9272
:10238000EF92FF920F931F93CF93DF930F92CDB7EE
:10239000DEB7EE24E394F12C0DE514E09E012F5FEF
:1023A0003F4F45E454E063E082E00E94CF10082FE5
:1023B000882321F1C09044048C2D90E09C01265983
:1023C0003B4F79011981F9018081181BD12E80E0E2
:1023D0000AC0DA94F70180818F5F808360E08C2DE2
:1023E0000E941B0B802F1D14A4F3912F17FD90E06A
:1023F000191B11110EC081110E945909802F0F90D5
:10240000DF91CF911F910F91FF90EF90DF90CF90D0
:1024100008951F5FF70180818150808361E08C2DDA
:102420000E941B0B802FE5CFCF93DF93CDB7DEB794
:1024300028970FB6F894DEBF0FBECDBF4091400481
:102440005091410460914204709143042FB7F89475
:102450008091520490915304A0915404B09155047A
:102460002FBF841B950BA60BB70B84369105A105D6
:10247000B105A0F10E942B0B882391F10E9439092C
:10248000462F572FBC014E5F5F4F6F4F7F4F4983E1
:102490005A836B837C8380914001909141018A5AD9
:1024A0009B4F20913F01422F50E0253010F044E037
:1024B00050E0BE016F5F7F4F0E941C2884E090E0D7
:1024C0000E941127892B19F50E9439096093400455
:1024D00070934104809342049093430481E018C0B8
:1024E0000E9439096D837E838F83988740916D04A4
:1024F00050916E0460916F04709170048D819E8183
:10250000AF81B885480F591F6A1F7B1FBCCF80E081
:1025100028960FB6F894DEBF0FBECDBFDF91CF91E6
:1025200008951F93CF93DF93982F162F81E09A3051
:1025300019F09D3031F480E0DF91CF911F910C9420
:102540002413C0910402D091050286E0FE01ABEF96
:10255000B1E001900D928A95E1F7903EA8F186E0F6
:10256000FE0111928A95E9F7C0910402D09105020B
:10257000111136C046E050E0BE018BEF91E00E94A1
:102580000F289E0127523240892BA9F52A5F3F4F21
:1025900040910602642F70E0C9010E94C527481BC4
:1025A000463010F4240F311D211572E0370710F06A
:1025B00030E020E0295D3D4F309305022093040276
:1025C000DF91CF911F910895F6E09F9FB0011124F4
:1025D0006D517E4F46E050E0CE010E940628C4CFE8
:1025E0009E012A5F3F4FFE012E173F0719F280819F
:1025F00080958193F9CFC90145E0969587954A95D5
:10260000E1F741E050E0BA0102C0660F771F8A95FA
:10261000E2F7CB016091290470912A04862B972B55
:10262000B9016B5F7F4FE5E076956795EA95E1F735
:1026300002C0440F551F6A95E2F7842B952B9093A7
:102640002A0480932904A2CFCF93E82F209104027B
:10265000309105022752324040910602642F70E00B
:10266000C9010E94C527481B842FEE2369F066E04C
:102670000E94D927C82FC15010F4CF91089560E06F
:1026800080E20E949112F7CFA901480F511D411518
:10269000524018F080E030E020E0280F311D295D25
:1026A0003D4F3093050220930402E7CF1F93CF9351
:1026B000DF93EC01162FFE018491811104C0DF919C
:1026C000CF911F910895612F0E9491122196F3CF0F
:1026D0000E94561381E00C942413CF92DF92EF9264
:1026E000FF920F931F93CF93DF936C017B0164E6FE
:1026F00070E088E70E949824EC018601EC0CFD1C38
:1027000097FD0EC0F801849164E670E00E941125E7
:10271000EC01892B29F40F5F1F4FE016F10691F7AA
:102720000E949E25CE01DF91CF911F910F91FF90C6
:10273000EF90DF90CF900895CF93DF9300D000D03B
:10274000CDB7DEB7809132048823F9F00E943909B1
:10275000DC01CB01805A9541AF4FBF4F80932B04D2
:1027600090932C04A0932D04B0932E0480912F04F9
:1027700081110BC062E070E080E491E00E946D1373
:10278000892B19F481E080932F040F900F900F9004
:102790000F90DF91CF9108951F921FB61F921124C1
:1027A0008F939F93AF93BF9380910102811113C0C8
:1027B0008091520490915304A0915404B091550417
:1027C0004196A11DB11D8093520490935304A09390
:1027D0005404B0935504BF91AF919F918F911F9076
:1027E0001FBE1F9018952FB7F894809152049091B6
:1027F0005304A0915404B09155042FBF08959C0137
:102800004FB7F8948091520490915304A0915404CE
:10281000B09155044FBF821B930B08959F92AF92C6
:10282000BF92CF92DF92EF92FF920F931F93CF93BD
:10283000DF93CDB7DEB763970FB6F894DEBF0FBE58
:10284000CDBF1A821982FE01339688E0DF011D9206
:102850008A95E9F782E9C82E81E0D82E8E010F5FB4
:102860001F4F5801EE24E394F12CF60181916F0182
:102870008F3F09F447C0F894E82FE295EF70F0E03D
:1028800021A18F70A70102C0440F551F8A95E2F75E
:10289000CA01922F982B91A392A18095892382A39C
:1028A000789400C0ECE9F1E030E020E0912C8191D7
:1028B0008F3F09F469C0A82FA295AF70A05EB0E069
:1028C0004C9150E08F7002C0559547958A95E2F77C
:1028D00040FD5AC08E2D022E01C0880F0A94EAF7DF
:1028E000982A2F5F3F4F2630310509F7F6013197BF
:1028F00080818F3F11F00E94000850EA5A95F1F74D
:10290000D8019C920F5F1F4FB7E9CB16B1E0DB06F1
:1029100009F0ABCF4AE050E0B50181E894E00E94B5
:102920000F288C01892B41F08AE0F501A1E8B4E081
:1029300001900D928A95E1F7F09080040115110540
:1029400029F181E0809366040E94F313909365045B
:102950008093640480916404909165040E94FF1345
:10296000059768F0AF2DB0E0AA58BB4F85E0E1E8CD
:10297000F4E001900D928A95E1F710926604012B24
:1029800049F081E090E066C080E0AACF80916604C3
:102990008111E0CF0E942B0BF82EE0918004882358
:1029A00009F490C01C861B869E01235F3F4F83E085
:1029B000D9011D928A95E9F70E2F10E00A581B4F96
:1029C000809167048A3008F057C06E01BBE0CB0EDF
:1029D000D11C21E831E14BE451E0B601C8010E946D
:1029E0005E0BBC2CED2C882309F45BC02EEB31E18F
:1029F00048E551E0B601C8010E945E0B882309F446
:102A000050C024E132E140E651E0B601C8010E9425
:102A10005E0B882309F445C010926704E0917504A9
:102A2000F0E0BF016A587B4FAB2DBE2D9E01205FA9
:102A30003F4F90E0FB014191BF018D91481731F06C
:102A4000AF0141505109FA0180839F2D2A173B079E
:102A500089F7892F63960FB6F894DEBF0FBECDBFFE
:102A6000DF91CF911F910F91FF90EF90DF90CF906A
:102A7000BF90AF909F9008958091680490916904F1
:102A80000E94FF13843F914008F09FCFE0917504AE
:102A9000F0E0EA58FB4F85E0DF011D928A95E9F7E7
:102AA00070CF909167049F3F31F09F5F90936704D0
:102AB0009A3008F4B3CF0E94F31390936904809383
:102AC0006804E4CFF0E0EA58FB4FF89485E0A7E50E
:102AD000B4E001900D928A95E1F765E070E087E53A
:102AE00094E00E941908809356047894F894E09139
:102AF0006C04F0E0E659FB4F80818B8780935D0486
:102B000061E070E0CE010B960E94190880935C048E
:102B10007894F894C0905E04D0905F04E0906004D4
:102B2000F09061048091710490917204A0917304FB
:102B3000B0917404C816D906EA06FB06F1F0C092FB
:102B40007104D0927204E0927304F09274040E94B3
:102B50002B0B811112C00E943909688B798B8A8BEB
:102B60009B8BC61AD70AE80AF90AC0926D04D09264
:102B70006E04E0926F04F0927004789480E06ACF63
:102B8000FF920F931F93CF93DF93C62FD42F122F53
:102B90008823A9F06093A6040E94F3139093DE01AA
:102BA0008093DD01C77081E001C0880FCA95EAF704
:102BB000DF91CF911F910F91FF900C94230680918C
:102BC000A604681334C08091DD019091DE010E945B
:102BD000FF138436910558F500E20D0FCD17A9F0CB
:102BE000C770FF24F3948F2D01C0880FCA95EAF7B0
:102BF0000E942D06083048F48D2F877001C0FF0C0D
:102C00008A95EAF78F2D0E942306812F0E94FF0AE2
:102C10000830A0F4D77081E001C0880FDA95EAF798
:102C2000DF91CF911F910F91FF900C942D06C770EB
:102C300081E001C0880FCA95EAF7F2CFDF91CF910A
:102C40001F910F91FF9008953F924F925F926F9264
:102C50007F928F929F92AF92BF92CF92DF92EF922C
:102C6000FF920F931F93CF93DF9300D000D0CDB787
:102C7000DEB77C01FC019081818123813481232B8B
:102C800021F089238F3F09F0EEC40F900F900F9031
:102C90000F90DF91CF911F910F91FF90EF90DF90F8
:102CA000CF90BF90AF909F908F907F906F905F90EC
:102CB0004F903F900895980122513F4520313105B2
:102CC00008F07DC48FEF93E00E942528025137E081
:102CD000832E32E0932E882369F18091AE048770B1
:102CE000A1F2F7018281882381F282E00F900F9098
:102CF0000F900F90DF91CF911F910F91FF90EF9068
:102D0000DF90CF90BF90AF909F908F907F906F900B
:102D10005F904F903F900C94B7088114F4E09F06A9
:102D2000E1F2C4010E942528811101C001502FEF5A
:102D3000821A920A0111F1CF8091470190914801C6
:102D4000A0914901B0914A0189839A83AB83BC83E6
:102D5000442443942AE0322E84010F5F1F4FC401A4
:102D60000E94252889831A82882309F4B6CF9FEF11
:102D7000980F9330F8F48A83498232E0830E911CD5
:102D8000C8010E9425288B83882309F4A6CF8E01D1
:102D90000F5F1F4FF80120812223F1F29181213032
:102DA00009F044C08281913039F40E5F1F4F0E94B8
:102DB000FF0A08C04801EBCF923039F40E5F1F4F75
:102DC0000E94ED080F5F1F4FE5CF933029F40E5F8F
:102DD0001F4F0E945B08F6CF943019F00F5F1F4F12
:102DE000F1CF0E5F1F4F20E030E0B8016F5F7F4FE3
:102DF000F80141818053990B8A30910560F02115CB
:102E0000310501F38FE99FE00197F1F700C0000061
:102E100021503109F4CF329EF001339EF00D112480
:102E20009C012E0F3F1F842F8B01DFCFE22FF0E09C
:102E3000EF52F64F5490822F86958695869590E0B6
:102E4000FC01EF53F64FE4912770F0E0022E02C030
:102E5000F595E7950A94E2F73F0131E06322772484
:102E6000FC01EF54F64FA490B12C022E02C0B59491
:102E7000A7940A94E2F7E1E0AE22BB24FC01EF55EF
:102E8000F64FC490D12C02C0D594C7942A95E2F78E
:102E9000F1E0CF22DD246114710419F081EE0E946B
:102EA000ED08A114B10419F086EE0E94ED08852DFD
:102EB0000E94FF0AAB2819F086EE0E945B08672883
:102EC00019F081EE0E945B08CD2809F47BCF8CE2DB
:102ED0006ECF81E00E94A0080E94630AFECE81E0CE
:102EE0000E94AB08F9CF82E0F5CF053F2CE5120731
:102EF000D1F027E245EE66EE063F3CE5130741F0D0
:102F000027E245EE64EE043F9CE5190709F07CC317
:102F10000E94C015E2CE27E245EE65EEF9CF26E22B
:102F200041EE60EEF5CF26E241EE62EEF1CF980180
:102F30002A5F3C452930310508F475C306319CE50C
:102F4000190709F0C8C09091A804882309F4B9C0F2
:102F5000892F8A7A91E009F490E09093A70469E2BE
:102F6000811165E385ED91E00E94D3080E94F6058A
:102F7000B4CEF801E350FC458091AC048160E331AC
:102F8000F105B8F4ED58F74D0C94F927C8018A5FA4
:102F90009C45099708F057C3F801EB5FFC45E83002
:102FA000F10590F4EA57F74D0C94F9278091AC04A1
:102FB00082608093AC0447C38091AC048460F9CFF5
:102FC0008091AC048860F5CF8091AD0481608093DE
:102FD000AD0439C38091AD048260F9CF8091AC0417
:102FE0008061E7CF8091AC048062E3CF8091AC0434
:102FF0008064DFCF0E94990D8091AC048068D9CFA6
:103000008091AC048C60D5CF8091AD048360DFCF1C
:103010008091AC048E7FCDCF8091AC048D7FC9CFE1
:103020008091AC048B7FC5CF8091AC04877FC1CFEA
:103030008091AD048E7FCBCF8091AD048D7FC7CFC3
:103040008091AC048F7EB5CF8091AC048F7DB1CFE1
:103050008091AC048F7BADCF0E94990D8091AC0420
:103060008F77A7CF8091AC04837FA3CF8091AD04ED
:103070008C7FADCF8091AC0482FB992790F921E041
:10308000922790FB82F990FB83F993CF8091AD0456
:10309000982F909591708E7F892B90FB81F997CF17
:1030A0000E94990D9091AC04892F97FB87F9805865
:1030B00080CF61E08EE090E00E943328C4C260E0DF
:1030C000F9CF8091A704811104C089E20E94E30531
:1030D0004DCF85E3FBCF0A35EDE51E0709F48FC020
:1030E00008F06BC001152CE5120709F478C00E3DFD
:1030F0001C4509F481C0F7018281C080D1808823FA
:1031000009F481C0C6010E94100D182F682FC60156
:103110000E948205B601812F0E94030D0E947B064A
:103120008C01F701B280A580A2949FE0A922809132
:10313000AE048770A1F0CB2CBB2091F0812F807F53
:10314000803421F080E2800F883048F082E00E94D5
:10315000B7088091AE048770CC24C3948111C12C30
:10316000D12ED2948FE0D822F8E0DF1609F43BC1CB
:10317000FD1508F489C023E02D1508F449C0812FFE
:10318000807F1F7031E03D1508F091C0803211F052
:103190001295107F002309F4C4C0013009F4E6C081
:1031A000BB2009F4F0C0AA2009F4E6C0F70185812C
:1031B00080FF92C08F708583DFC00B358DE51807C7
:1031C00001F10C351D4509F096CF8091AD0482FBCD
:1031D000882780F991E089270E94050C8CCF0E94F6
:1031E000990DEFEFF4E32CE0E150F0402040E1F7DF
:1031F00000C000000E945B090E9465106ECD81E056
:10320000EBCF80E0E9CFC6010E94B005182F82CF36
:1032100084E0D81609F4CDC02D2D2850330B24306E
:10322000310510F40E944E0BCC20A9F08091AE0421
:1032300080FD11C0F70112828595859585950E94C4
:10324000A008C7010E9424168091AE04859585953B
:1032500085950E94AB0860E0C7010F900F900F901A
:103260000F90DF91CF911F910F91FF90EF90DF9022
:10327000CF90BF90AF909F908F907F906F905F9016
:103280004F903F900C943F0D99E0D91609F41BC163
:1032900086E08D0D8F70823008F0BECF023F09F0BE
:1032A00021C1812F8F71BB2009F45CC118C1882313
:1032B00011F01295107FBB20C9F0112369F080E254
:1032C000800F883010F001110BC08091A804812B71
:1032D0008093A8040E94F605802F0E94ED089CCFE1
:1032E0008091AF04812B8093AF04F4CF802F0E9494
:1032F0005B08112309F490CF109580E2800F88308D
:1033000010F0011108C08091A80481238093A804C3
:103310000E94F60581CF8091AF0481238093AF0492
:10332000F7CFBB20B1F09091A904812F892BA11078
:1033300003C00E94230670CFE1E0AE12FACF2091C5
:10334000AD0422FD69CF981709F466CF8093A904D4
:1033500063CFA11006C00E94F005812F0E942D06A8
:103360005BCFF1E0AF1609F457CFF5CFBB2031F0BA
:1033700025E02A1508F450CF812FDBCF34E03A1531
:1033800008F44ACFEACFAA2041F3093369F4FFEFEA
:1033900027EE33E0F15020403040E1F700C000005C
:1033A000802F0E945B0838CF8FE39CE90197F1F7EB
:1033B000F5CF812F86958695837061F0813009F075
:1033C0002BCFC8019370B11002C090E080E00E9442
:1033D000450822CFC8019370B11002C090E080E090
:1033E0000E942F0819CF812F8370A1F5B11014CF3F
:1033F000802F829586958770880F880F402F4F7099
:10340000082E01C0440F0A94EAF7202F207104FF10
:1034100007C02FE030E001C0220F8A95EAF720951F
:10342000169516951370123081F0822F842B13306D
:1034300031F08091AA04113029F0242B82230E94BC
:103440009808EACE842B822BFACF242B8091AA04F1
:103450008227F5CFBB2061F110FFDECE802F829551
:1034600086958770880F880F402F4F70082E01C0F7
:10347000440F0A94EAF7202F207104FF07C02FE0C1
:1034800030E001C0220F8A95EAF72095169516952F
:103490001370123099F0822F842B133031F0809109
:1034A000AB04113041F0242B82230E949C08B4CE3F
:1034B00011FFB2CED3CF842B822BF7CF242B809158
:1034C000AB048227F2CF1F70BB2029F0812F0E940E
:1034D000A008802F2ECF802F0E942D06812F0E94C2
:1034E000AB089ACE033F60F4003F09F1013FA9F118
:1034F000BB2009F450C0A110EFCE812F8F7132C0D4
:10350000033F99F1043FA1F7BB20D1F11F71812F37
:103510000E94A0088091AD0482FD07C0F8E01F9FC3
:10352000C001112483608093AE04812F1BC0BB2097
:1035300079F094E09A1508F46FCE1F7181E090E065
:1035400001C0880F1A95EAF79091AB048927ADCF97
:10355000E5E0EA1508F460CEF0CF812F8F71BB2033
:1035600009F4BDCF0E94A00857CE80E0BB2009F42B
:103570009CCF1F7181E001C0880F1A95EAF795CFA3
:1035800081E00E94B70821E02A1508F045CE82E0CC
:103590000E94B70841CEAA2079F0093341F43FEFE9
:1035A00087EE93E0315080409040E1F7F7CEEFE3B3
:1035B000FCE93197F1F7F2CE812F8F7190CF003176
:1035C000FFE51F0709F485CC01312FE5120709F447
:1035D0008ACC033F2CE5120709F4A1CC08F085CC76
:1035E000083D9CE5190709F496CC28E241E0093D25
:1035F000ECE51E0709F491CC26E241EE61EE073DB1
:10360000FCE51F0709F484CC882309F441C010921B
:10361000A6040631ECE51E0708F089CC0230FCE573
:103620001F0708F45FCD0E94B60C9093AD04809301
:10363000AC0406312CE5120708F0A8CC02303CE5BA
:10364000130708F096CC6091AC041091AD0484E0AF
:1036500090E00E943328612F82E290E00E9433289C
:103660000E94990D3ACB61E0C7010E943F0D8C0189
:10367000F701828181111FCB00313FE5130709F467
:103680002ECC01319FE5190709F0A3CF82E028CCA9
:1036900006311C4509F457CC2ECD1F93CF93DF93F1
:1036A0008091E704807FA9F48091E404882389F065
:1036B0008091B104C091B0047091E2046091E30480
:1036C000A091E504B091E604D62FD72316E0C813E5
:1036D00004C0DF91CF911F91089590E0109711F0F1
:1036E000DF3F19F401968770F2CF189F9001199F60
:1036F000300D1124F901EE54FB4F41816413F2CFD8
:1037000040814713EFCF42814111ECCF4381548177
:103710004A1B5B0B4436510528F78091E7048F70F4
:1037200080618093E704F901E954FB4F80818F7039
:103730008061808382EE94E00E942416DF91CF9115
:103740001F910C94D9058F929F92AF92BF92DF92F6
:10375000EF92FF920F931F93CF93DF93CDB7DEB716
:103760002B970FB6F894DEBF0FBECDBF8C0185E05E
:10377000F801DE01179601900D928A95E1F7F801A4
:10378000E280A380B48082EE882E84E0982E90910F
:10379000E2048091E3042091E5043091E6042115D0
:1037A000310529F0482F49234F3F09F028C1EE2069
:1037B00009F433C1F801808191810E946C0DF82ECB
:1037C000882309F42AC186E0F801A2EEB4E0019052
:1037D0000D928A95E1F70E944D1B21C0D090E7041D
:1037E0004D2D407F2436310508F0A8C0F801218115
:1037F0004111C3C0FE2C281325C08081891322C02B
:10380000E11020C08D2D8F7080618093E70482EEDF
:1038100094E00E9424168091E704F80185838F2D9F
:103820002B960FB6F894DEBF0FBECDBFDF91CF91C0
:103830001F910F91FF90EF90DF90BF90AF909F90FE
:103840008F9008953F81AB2829F0822F83238F3FEB
:1038500009F090C080E0F82FF170DF2EE091B10404
:103860004091B00456E080FD1CC0EE20C1F2809172
:10387000E70481608093E704F12CD1CF8E2F90E094
:103880005E9FF0011124EE54FB4F6181261306C0A8
:103890006081361303C06281E612E7CF0196E82FFC
:1038A000E770E413EBCF8F8198850E945E0D292F7E
:1038B00022952F70903260F0225F2F70223078F4C2
:1038C0009F7051F0F8019581907F31F4D12C0AC09E
:1038D0009F7011F08823D1F3805E8830B8F3C8015F
:1038E0000E942416FD2C9BCFF801808191810E94BB
:1038F0006C0D882309F491C0EE2009F48EC08091EC
:10390000E704803270F08091E2049091E3049A839E
:1039100089831B82BD82AC82DE82CE0101960E9429
:10392000241686E0F801A2EEB4E001900D928A958B
:10393000E1F70E944D1BFF24F39471CF411132C077
:1039400082EE94E00E94241686E0F40111928A959A
:10395000E9F792CFF801808191810E946C0D81116D
:10396000E0CF8091E70481608093E704C8010E9462
:10397000241655CF81E08E256ECF2813B5CFF801E0
:1039800080818913B1CFE110AFCFD582C8010E94E9
:10399000241686E0F801A2EEB4E001900D928A951B
:1039A000E1F73DCFF801218182139ECFF80180819C
:1039B00089139ACFE11098CFD582C8010E942416AE
:1039C00086E0F40111928A95E9F729CFF801218167
:1039D0008213C0CFF80180818913BCCF8091E704A6
:1039E00080FDD7CF982F907FA1F28583903F71F211
:1039F000982F907F905F8F70892B8583C7CFF09031
:103A0000E404A501421B530B9A01F110E7CE2436C2
:103A10003105B0F6FE2CE110D9CFC8010E94241662
:103A20008ACF1F93CF93DF93CDB7DEB767970FB6DB
:103A3000F894DEBF0FBECDBF342F4B8B252F5C8B90
:103A4000962F6D8B7E8B8F8B4E895F8961111092C3
:103A5000AF041A8A3D872E879F87598B488B86E053
:103A6000FE013D96DE01179601900D928A95E1F7D1
:103A7000CE0107960E94A31B882389F016E080914F
:103A8000B1049091B004891349C067960FB6F894B9
:103A9000DEBF0FBECDBFDF91CF911F91089586E0AD
:103AA000FE013796DE01119601900D928A95E1F79D
:103AB0009F8188852091B0044091B1046A857B85FF
:103AC000672BE1F289238F3FC9F230E0C9010196EB
:103AD000877099274817190671F40E94990D109262
:103AE000B0041092B10486E0E2EEF4E0DF011D9232
:103AF0008A95E9F7C3CF96E0929FD001939FB00DCE
:103B00001124AE54BB4FFE01319601900D929A954F
:103B1000E1F78093B0040E94D905B0CF819FC00126
:103B200011248E549B4F0E94A31B882309F4ADCF10
:103B30008091B10490E00196877099278093B10439
:103B40009ECFCDB7DEB7A4970FB6F894DEBF0FBEF9
:103B5000CDBF84B7877F84BF0FB6F894A8958091B6
:103B60006000886180936000109260000FBE80E862
:103B700090E00FB6F89480936100909361000FBEBF
:103B800085B7806885BF85B7806885BF8EEF97E071
:103B90009093D3018093D2010E941A0A0E949E0A38
:103BA0008091E20084608093E200789480916204C6
:103BB000882399F08091E9001091EC001795112766
:103BC00017958F70182B1092E9008091E80083FD03
:103BD0000E94A40D1F701093E90082E084BD93E061
:103BE00095BD9AEF97BD80936E0010926D04109270
:103BF0006E0410926F04109270040E94C40C811124
:103C000002C00E94A70C0E942B0B809301010E940E
:103C10002B0B81110E9403268091010180910101EB
:103C200095E0811190E09093800485E0891B80935A
:103C3000750402E911E037E9E32E31E0F32ED801F3
:103C40008D918D018F3F11F00E940008E016F10662
:103C5000B1F70CE911E022EAE22E21E0F22EF801A0
:103C600081918F018F3F11F00E940008E016F1064C
:103C7000B1F78AE0E1E8F4E0DF01682E1D926A9472
:103C8000E9F7E6E7F4E0DF011D928A95E9F790E0B5
:103C900080E00E942D28893E9E4F21F40E94C40C92
:103CA000811102C00E94651082E090E00E942528E8
:103CB000809334040E94B60C9093AD048093AC04BE
:103CC0000E940E14EFE3FCE93197F1F700C0000009
:103CD0000E940E148091760480FF08C06FEF7FEF82
:103CE00090E080E00E9451280E945B0983E090E010
:103CF0000E9425280E9498080E942B0B811102C067
:103D00000E9406260E942B0B8111B6C090E080E82D
:103D100090932704809306020E9492246DE070E045
:103D200086E199E00E946D13892B09F043C08091D0
:103D3000270463E070E081FDA2C083E199E00E9466
:103D40006D13892BB9F56DE070E083E099E00E9476
:103D50006D13892B79F50E94390969A37AA38BA386
:103D60009CA3DC01CB01805A9541AF4FBF4F80939C
:103D70002B0490932C04A0932D04B0932E04E7E21F
:103D8000F2E080E092E0DF019C011D922150304082
:103D9000E1F7F0930502E09304028FEF9FEF909319
:103DA0002A048093290481E08093320480932F04B5
:103DB0001092280480910101811106C084EF809344
:103DC0000D0185EF80930C0140910D01A42FA29568
:103DD000AF70B0E091963C9191974F7081E090E088
:103DE000BC01042E01C0660F0A94EAF7262F209525
:103DF000232391962C93919792962C919297262B10
:103E000092962C93929730910C01E32FE295EF70EC
:103E1000F0E021A13F70032E01C0880F0A94EAF759
:103E2000982F9095922391A392A1892B82A390968B
:103E30002C9180A190E002C0959587953A95E2F784
:103E40008170880F30E002C0359527954A95E2F7DA
:103E50002170822B809303029091010181E09827C9
:103E600090936C04891B8093440482E091E09093CA
:103E70008C0480938B04EBC193E080E249CF80E116
:103E800099E05DCF80916204843021F110920102AB
:103E900048E150E080E40FB6F894A89540936000A4
:103EA0000FBE8093600083B7817F846083BF83B738
:103EB000816083BF7894889583B78E7F83BF0FB668
:103EC000F894A895809160008861809360001092BA
:103ED00060000FBE80913F04882361F00E940E14A1
:103EE000E6E7F4E081918111BBC3A0E8B4E0AE172E
:103EF000BF07C1F780916204853009F4C3CF0E94E7
:103F0000990D0E944E0BAAC1C394FF0C96E0692E36
:103F1000C610BAC10F5F1F4F0A30110509F0AAC1C0
:103F20008FEF89838A831B820E94F3138160782F2D
:103F30009D838C8349815A816B81892F0E94111D39
:103F4000C4C10E94F313909331048093300487E23C
:103F500092E090930502809304020E942B0B60E094
:103F6000882309F455C08CE599E00E94561380918E
:103F7000AB040E947205882341F0813021F160E09A
:103F80008DE499E00E94561305C060E087E599E052
:103F90000E94681360E08AE499E00E94561360E092
:103FA00084E499E00E9468138091AB040E9472053A
:103FB000823031F160F0833039F160E08CE299E0D9
:103FC0000E94681309C060E082E599E0E1CF60E0FB
:103FD0008EE399E00E94561360E089E299E00E9426
:103FE00056130E944E0B81FB662760F983E299E02D
:103FF0000E94681380913204882309F4E3C1DAC176
:1040000060E088E399E0E6CF60E082E399E0E2CF08
:104010008FE599E00E945613EDCF8091280461E06E
:1040200070E08111CFC1082F10E02B01082E02C0D3
:10403000440C551C0A94E2F7A90144215521452B53
:1040400009F44AC020912704922F917020FD46C0A8
:10405000980136952795369527958295880F807615
:104060003FE1380F80931001209313013093110129
:104070009093140124E630E047E050E06EE071E0F8
:1040800088E70E944025892B09F09CC1A80175E0B2
:10409000440F551F7A95E1F78091270480FD26C0D3
:1040A000495D5D4F04E610E020E230E060E488E71F
:1040B0000E946D25892B09F085C10E949C134094B4
:1040C00050948091290490912A0484219521909301
:1040D0002A048093290476C18F5FA5CF880F880FAB
:1040E000880F37E0380F20E093E0BCCFE7E0F2E044
:1040F00080E2DF011D928A95E9F70EE811E06AE897
:10410000C62E61E0D62E77E099249394D801ED91E4
:104110008D01D6018D916D01840F952F911D9C010C
:10412000295D3D4F1901F0E0E95FFD4F30E020E0EF
:10413000772E721A892D022E01C0880F0A94EAF791
:10414000510160E0D5019D915D019823A72DA61B2B
:10415000A7708A2E0A2E000CBB0B692E01C0660CBC
:104160008A94EAF7B195A195B109A770BB2701C060
:104170009695AA95EAF79629A0819A2B90836F5F6E
:10418000683001F72F5F3F4F31962830310581F6B7
:1041900022E931E02017310709F0B8CF04E610E03A
:1041A00020E230E047E052E081CF8091F100D80179
:1041B0008D938D01B1E0EB1AF10809F45DC1809196
:1041C000E80085FDF2CF8091E8008B778093E800CE
:1041D0000E94E909882399F34FC11A8289E08B83F1
:1041E00012C08A81823009F451C2833009F456C169
:1041F000813009F071C10E9439090E94FF276B8349
:104200007C838D839E8380916204843001F580914C
:10421000E9001091EC001795112717958F70182B56
:1042200082E08093E9008091E80080FF0DC050E0BB
:1042300040E060E270E0CE0101960E94390A809170
:10424000E8008E778093E8001F701093E90080915A
:10425000620400E112E1853009F44CCE0E940E1494
:10426000E82E81110E943909A6E7B4E0E5E3F4E005
:1042700010E000E0B02EDD9081918D1509F44ACE5A
:104280008D25C12CFF24F394982F9F2109F43CCE57
:104290000E942B0B882399F0C982BA82DF2081E02B
:1042A00009F480E08B830E94F3138160782F9D8353
:1042B0008C8349815A816B81892F0E94111DF801DD
:1042C000EB5CFB4F80818F25808340910D01E42FB3
:1042D000E295EF70E05EF0E0208130910C01E32F79
:1042E000E295EF70E05EF0E0808190E03F7002C008
:1042F000959587953A95E2F7880F991F82709927CF
:1043000030E04F7002C0359527954A95E2F721704D
:104310003327822BE0910302EE0FEE0FE82BE093A0
:10432000030210916C04EF70F0E0E658FE4F8081BC
:1043300090910202890F80930202F12C82306CF07E
:10434000E12FF0E0E659FB4F80818F5F808360E0D2
:10435000812F0E941B0BFF24F394809102028F3F58
:104360006CF4E12FF0E0E659FB4F808181508083AF
:1043700061E0812F0E941B0BFF24F39480910202C5
:10438000082E000C990B62E070E00E94E5278093F4
:104390000202F1100E94590980913204882309F425
:1043A00040C080913004909131040E94FF13C29765
:1043B00008F0C7CD2091290430912A042115310538
:1043C00009F02BCE80912F04882359F10E943909DE
:1043D00069A37AA38BA39CA380912B0490912C04B6
:1043E000A0912D04B0912E0429A13AA14BA15CA16A
:1043F000281B390B4A0B5B0BDA01C9018F3F9F4F1A
:10440000AF4FBF4770F480913204882351F062E0CF
:1044100070E08FE999E00E946D13892B11F41092DE
:104420002F04E11001C0F1100E949C130E944E0B5A
:1044300090913304891721F00E944E0B809333042E
:1044400080916204843009F002CF83E08093E90018
:104450008091E80082FFFBCE8091E80090E085FF2C
:104460000CC00E94E90950E2E52EF12C8E010F5F8D
:104470001F4F882309F4A3CE91E08091E8008B7749
:104480008093E800992309F4E2CEE981E150E33119
:1044900018F5F0E0E257F74D0C94F9278AE0E6E7CB
:1044A000F4E0DE01139601900D928A95E1F7ABCE10
:1044B0008A81823089F42B813C814D815E8129A3E0
:1044C0003AA34BA35CA3CA01B9010E94FF2786E26D
:1044D00090E00E94332897CE8FEF898394CE4C8151
:1044E0006B818A810E94DD0C9827892798279E83FB
:1044F0008D8389CE0D811E811027012710278A8187
:10450000EB803CE0E39E7001112448E7849FE00CBF
:10451000F11C11248C8190E0880F991FE80EF91E80
:10452000612FC70187960E943328602FC7018896A4
:10453000D0CF0E941F0C67CE80E18A8364CE81E0D9
:104540008A8389EF4CCECA80DB80DC24CD24DC2436
:104550008C817601E80EF11C8E010B5F1F4FC601A6
:10456000895F9D4FCE14DF0409F44DCE59EFC51677
:1045700051E0D50648F40E942528D8018D938D017D
:10458000BFEFCB1ADB0AEBCF80E0F7CF0A811B81AC
:10459000102701271027FE0131966F018C817F01C2
:1045A000E80EF11CC801895F9D4FCE14DF0409F4A9
:1045B0002ACE093FF1E01F0728F4D60114966C912A
:1045C0000E9433280F5F1F4FBFEFCB1ADB0AEACFE1
:1045D0000E94970C18CE84E0B0CFCA80DB80DC2428
:1045E000CD24DC248C817601E80EF11C8E010B5F5A
:1045F0001F4FC6018796EC14FD0409F404CEE0EECB
:10460000CE16E1E0DE0648F40E942528D8018D93FD
:104610008D01BFEFCB1ADB0AECCF80E0F7CF0A8128
:104620001B81102701271027FE0131966F018C8115
:104630007F01E80EF11CC8018796CE14DF0409F44F
:10464000E2CD003EF1E01F0728F4D60114966C91EC
:104650000E9433280F5F1F4FBFEFCB1ADB0AEBCF4F
:1046600009BD19BD09B400FEFDCF8091D8008F7D32
:104670008093D8008091E00082608093E000809178
:10468000E00081FDFCCF0E94990D34CC86E290E0E1
:104690000E9425281B821C821D828E83B4CD7894B3
:1046A0001F921FB61F9211248F939F93AF93BF93B6
:1046B0008091520490915304A0915404B0915504F8
:1046C0000196A11DB11D8093520490935304A093B1
:1046D0005404B0935504BF91AF919F918F911F9057
:1046E0001FBE1F9018951F920F920FB60F921124A4
:1046F0002F933F934F935F936F937F938F939F93EA
:10470000AF93BF93EF93FF938091E10082FF09C0C5
:104710008091E20082FF05C08091E1008B7F809351
:10472000E1008091DA0080FF24C08091D80080FFF2
:1047300020C08091DA008E7F8093DA008091D900CA
:1047400080FF99C080E189BD82E189BD09B400FE86
:10475000FDCF81E0809362048091E201811109C064
:104760000E941A0A0E949E0A8091E200846080934F
:10477000E2008091E10080FF17C08091E20080FF9D
:1047800013C08091E2008E7F8093E2008091E2006E
:1047900080618093E2008091D80080628093D8008D
:1047A00019BC85E0809362048091E10084FF27C0FA
:1047B0008091E20084FF23C080E189BD82E189BD50
:1047C00009B400FEFDCF8091D8008F7D8093D80082
:1047D0008091E1008F7E8093E1008091E2008F7EE6
:1047E0008093E2008091E20081608093E2008091FA
:1047F000E101882309F445C084E08093620480913C
:10480000E10083FF27C08091E20083FF23C08091F5
:10481000E100877F8093E10082E080936204109240
:10482000E1018091E1008E7F8093E1008091E200C0
:104830008E7F8093E2008091E20080618093E200AD
:1048400042E060E080E00E946E0A8091F0008860A3
:104850008093F000FF91EF91BF91AF919F918F9165
:104860007F916F915F914F913F912F910F900FBE6C
:104870000F901F90189519BC109262041092E201DB
:1048800078CF8091E30087FD02C081E0B6CF83E05E
:10489000B4CF1F920F920FB60F921124FF920F9375
:1048A0001F932F933F934F935F936F937F938F93B8
:1048B0009F93AF93BF93CF93DF93EF93FF9309EE53
:1048C00010E0F8018081C091EC00C795CC27C79516
:1048D0008F70FC2EF82A1082C0EFD0E08881877F8D
:1048E000888378940E94A40DF801108288818860E2
:1048F0008883CF2DCF70C083FF91EF91DF91CF914F
:10490000BF91AF919F918F917F916F915F914F91E7
:104910003F912F911F910F91FF900F900FBE0F901D
:104920001F9018951092B9008CE08093B8000895FC
:104930009F92AF92BF92CF92DF92EF92FF920F932E
:104940001F93CF93DF93B82EEB010E94F3136C01FA
:10495000EE24E394F12CC431D10560F025E0E22E81
:10496000F12CCF3FDC0731F0CE0164E170E00E9412
:10497000C5277B0184EAA82E94E8992E1092BC00EA
:10498000A092BC000E94F3138C018091BC0087FFB1
:104990000CC08091B900887F883031F18091B900D6
:1049A000887F803109F10FEF08C00E94F313801B4C
:1049B000910B8E159F0548F30EEF1FEFCF3FDC07DD
:1049C000E9F2C6010E94FF138C179D07B8F2C801D7
:1049D000DF91CF911F910F91FF90EF90DF90CF90DB
:1049E000BF90AF909F900895B092BB009092BC0092
:1049F0000E94F3138C018091BC0087FF0AC02091B4
:104A0000B900287F283111F0203469F600E010E069
:104A1000DECF0E94F313801B910B8E159F0558F378
:104A2000CBCF0F931F93CF93DF93EB018093BB000A
:104A300084E88093BC000E94F3138C018091BC0039
:104A400087FF11C02091B900287F81E090E02832D3
:104A500011F490E080E0919581959109DF91CF91DB
:104A60001F910F910895CF3FDC0741F30E94F3138C
:104A7000801B910B8C179D0708F38EEF9FEFEECFF5
:104A8000CF92DF92EF92FF920F931F93CF93DF931A
:104A90006B018A01F22EE32E622F732F0E9498245D
:104AA000AC01E6010C0D1D1DC017D10711F057FF19
:104AB0000DC084E98093BC00CA01DF91CF911F91A2
:104AC0000F91FF90EF90DF90CF9008956F2D7E2D86
:104AD00089910E941125AC01E7CFCF92DF92EF922E
:104AE000FF920F931F93CF93DF93C62F6A01790133
:104AF000B8010E9498249C0197FD0DC0B8018C2F2D
:104B00000E9411259C01E601EC0CFD1CCE15DF0571
:104B100011F037FF0DC084E98093BC00C901DF911B
:104B2000CF911F910F91FF90EF90DF90CF9008955C
:104B3000B80189910E9411259C01E8CF84E98093F6
:104B4000BC0008958EE14A9B02C08150E1F74A9B68
:104B5000FECF08955A9880E28A95F1F75A9A0895FF
:104B6000FC013BE03A95F1F798E020E080E031E08D
:104B700040E14A95F1F7880F4A9B02C081602327E4
:104B800042E04A95F1F7000040E14A95F1F7915073
:104B900079F790E19A95F1F799B132E03A95F1F70A
:104BA000000040E14A95F1F792FB992790F992278E
:104BB0002081920F90830895EF92FF920F931F939D
:104BC000CF93DF930F92CDB7DEB719828C017C01B2
:104BD000E60EF11C0E151F0561F481E0998191111B
:104BE00080E00F90DF91CF911F910F91FF90EF9098
:104BF00008950E94A225CE0101960E94B025F801D9
:104C000081938F01E7CF529A5A9A089552985A9AEF
:104C1000EA9AE9E6F0E080818F7C80830895615014
:104C2000770B91E001C0990F6A95EAF720E031E037
:104C3000911108C0222391F05A9A80E28A95F1F7E7
:104C40005A980895492F482339F05A9A232740E269
:104C50004A95F1F79695ECCF5A98F9CF5A98EDCF3F
:104C6000FF920F931F93CF93DF93EC018C01060FFC
:104C7000111DC017D10731F4DF91CF911F910F9112
:104C8000FF900895F9900E94AA2568E08F2D0E9458
:104C90000F26EFCF1F920F920FB60F921124EF92B3
:104CA000FF920F931F932F933F934F935F936F93B5
:104CB0007F938F939F93AF93BF93EF93FF93CF9384
:104CC000DF930F92CDB7DEB719820E94A225CE01E5
:104CD00001960E94B025282FA82FA695A695A695E7
:104CE000982F929595708A2F8570980F892F8370D1
:104CF00096959695890F822787709981892B09F05F
:104D000075C0A63008F072C080E18A95F1F75A9A12
:104D1000529AB2E0BA95F1F700C0EA2EF12C5A98F7
:104D2000EAE0AE9FD0011124AB5EBE4F1896ED9124
:104D3000FC9119973097B1F06091A2017091A30195
:104D400016962D913C911797260F371F13968D912C
:104D50009C911497680F791F15964C911597129690
:104D60008C9109958AE08E9DF0018F9DF00D1124A4
:104D7000EB5EFE4F6581662351F02091A2013091D8
:104D8000A30186819781820F931F0E9430260E9483
:104D9000AA25F0E1FA95F1F75A9852985A9A80E1CB
:104DA0008A95F1F78AE08E9D80018F9D100D112468
:104DB0000B5E1E4FD80112966C911297662371F10B
:104DC0002091A2013091A30113968D919C91820FA5
:104DD000931F0E94DC25D801ED91FC91882311F0EE
:104DE00088E001C082E080830E94A2250F90DF91BD
:104DF000CF91FF91EF91BF91AF919F918F917F9153
:104E00006F915F914F913F912F911F910F91FF9063
:104E1000EF900F900FBE0F901F901895ED91FC91A1
:104E2000DFCF0F931F93CF93DF93EC0106970CF026
:104E3000A9C08AE08C9FF0018D9FF00D1124EB5EDC
:104E4000FE4F80819181892B09F49CC0F894529A7D
:104E50005A9885E08A95F1F700008C2F8695857029
:104E60009C2F9570890F982F937086958695890F42
:104E70008E0193E0000F111F9A95E1F7082B0E9415
:104E8000AA2500C068E0802F0E940F26A0E1AA9505
:104E9000F1F752985A9A4A9B27C087E090E04A99C6
:104EA00025C08AE08C9F80018D9F100D11240B5E20
:104EB0001E4FF80165816623A1F12091A201309176
:104EC000A30186819781820F931F0E94DC258111A7
:104ED00028C0529A5A9AD801ED91FC9182E08083C1
:104EE000789482E090E016C000C0D5CF0197B9F465
:104EF000529A5A9A8AE08C9FF0018D9FF00D1124EE
:104F0000EB5EFE4F0190F081E02D81E0808378948C
:104F100081E090E0DF91CF911F910F91089500C043
:104F2000BECF0E94A225B0E2BA95F1F75A98529AE4
:104F3000E0E1EA95F1F78AE08C9FF0018D9FF00D9A
:104F40001124EB5EFE4F6281662351F02091A20195
:104F50003091A30183819481820F931F0E94302698
:104F60000E94AA258AE08C9FF0018D9FF00D1124EC
:104F7000EB5EFE4F0190F081E02D1082789490E07E
:104F800080E0C8CF84E090E0C5CFAA1BBB1B51E1F5
:104F900007C0AA1FBB1FA617B70710F0A61BB70BA9
:104FA000881F991F5A95A9F780959095BC01CD014E
:104FB0000895991B79E004C0991F961708F0961B75
:104FC000881F7A95C9F78095089597FB072E16F4E8
:104FD000009407D077FD09D00E94C52707FC05D0B3
:104FE0003EF4909581959F4F0895709561957F4F00
:104FF0000895EE0FFF1F0590F491E02D09946927A5
:10500000962769277827872778270895FB01DC01F1
:1050100002C005900D9241505040D8F70895FB0111
:10502000DC0104C08D910190801921F44150504061
:10503000C8F7881B990B0895FB01DC0102C00190A1
:105040000D9241505040D8F70895F999FECF92BD86
:1050500081BDF89A992780B50895A8E1B0E042E0B3
:1050600050E00C945928262FF999FECF92BD81BDAE
:10507000F89A019700B4021639F01FBA20BD0FB696
:10508000F894FA9AF99A0FBE08950396272F0E9472
:1050900034280E943328252F0E943428242F0C9472
:1050A00034280196272F0E9434280C943328DC01E1
:1050B000CB01FC01F999FECF06C0F2BDE1BDF89A23
:1050C000319600B40D9241505040B8F70895F894CD
:1050D000FFCF860EAE0E4D10AE0E4D10E10E020F3C
:1050E0004D10FE0F0B10D617DC17E017EE17F21756
:1050F000F617FA17001808180C18101814182018AA
:10510000241828182C18321850183A18EA171818AA
:105110001C1804183618461859185F18ED20F1208D
:1051200058226F227A2299226C226C226C226C22E5
:105130006C229C229F22A322C622E822EB22ED228F
:025140000F233B
:1051420001016C09A30B6F09FD0B010CF4F50021A1
:10515200007F220003D4010000000100000000D4FF
:10516200010000000501000000D40100000001065A
:10517200000000D4010000000107000000D4010477
:105182000800000000000000000000736C617665FA
:105192005F6D617472697800656E636F6465720039
:1051A20073796E635F74696D65720040223200012B
:1051B200DE00AC0054016D018D0100FF0100010011
:1051C20000FFFF0000010001FF0000081018181086
:1051D2000800946697C6340000000000313233366E
:1051E200F7F65604E200E900EA00B500B600B7009F
:1051F200CD008301CC008A01920194012102230295
:1052020024022502260227022A02B300B4006F00FC
:0252120070002A
:00000001FF
